:020000040000FA
:10000000640085018601C6289900030E9A00040841
:10001000AA001108AB009008AC00910190012B20C0
:10002000A0109318A0142D08840012088000AD0AB7
:100030002D08373C031928282B0891002C08900024
:100040002A0884001A0E8300990E190E8B100900DD
:100050002F30AD001C2805089B00831606089C0065
:100060000612861683120A308500061111084620F2
:10007000930010084620920006151F308500831655
:100080001C08860083121B088500080094000830B5
:100090009600940D06120318061686140310861A8D
:1000A0000314950D8610960B49281508080090003A
:1000B0008030230491002B20080083160F30860522
:1000C000831206080F39980E180486001708850059
:1000D00006110000000000000000000000000615EE
:1000E0001F30850008008316F0308604831217083D
:1000F00085000608F0399800980E1F30850008002A
:10010000890083168B138811081555308900AA3091
:10011000890088148B170811831208002D082E02FD
:10012000031985292E088400AE0A2E08373C031DCA
:100130009B282F30AE0000081F399E000008E039D0
:10014000A100A10E0310210C82073A2940294A2957
:10015000512957295A296029AD281E08EA3C03195C
:10016000B0281E1E84291E080F39820765296729B9
:1001700069296C296F297129732975298429842992
:1001800084297E29802977297C29B0288316850136
:100190000930860083120730A400A801A90120308D
:1001A000A600203089008316081483120808A200D4
:1001B000221DE8282030970097031708890083162E
:1001C00008148312080898005D209708031DDC2896
:1001D000A301E4309100023090002B2040309100C8
:1001E00090012B201208023C031DE8282F30AD009F
:1001F000AE008316810183120B168B17F530572042
:100200006400201C0629861D20101029861D102937
:1002100020140B309700732018080F3940385720EE
:10022000A21D8E28A50B8E28A60B8E282030A60096
:1002300014309700732098080314031D0310A80DB1
:10024000A403A41F342928082902031931292808E6
:100250000F3980385720280E0F39A038572028082A
:10026000A900A8010730A4000330970024089800D3
:100270005D208E281D0897007320180857205E29DE
:100280001D08890083160814831208081F392038B6
:1002900057205E291D0897000F301E0598005D202D
:1002A0005E2964001E0888001D0880205E291E0843
:1002B0009D005E291F081F3960385720221C8529A0
:1002C0001E081F39C038572085292210842922147E
:1002D0008429A210A3018429A214A3148429221121
:1002E000842922158429A2118429A215842922088F
:1002F000880020308020842988017929A9013129AA
:1003000022081F39203857205E290330A005031A20
:10031000201583168818A015881920168312200826
:040320009F00002911
:02400E00FD3F74
:10420000000000000000000008000800080008008E
:1042100001000700000000000F0004000B00000078
:10422000000000000000000000000000000000008E
:10423000000000000000000000000000000000007E
:024240000E006E
:00000001FF
